:100000003C2998181812181664008C1E04281A0827
:1000100003143729040864000C1E0B2899000314EC
:10002000372964002720031811289A20A8010830D6
:10003000A3009B2027200318A80AAB1EA801A20C2E
:10004000A30B1928AB1AA2139B20220808003A0818
:100050008400380884178004841300052B1B38069D
:10006000FF3E0800A401A501B7123221D33E0319B7
:10007000B7162D3EC63E031835280A3E031C352808
:10008000A2000310240DA000250DA100200DA10D3C
:10009000A4070318A10A2108A507A40DA50D22088D
:1000A000A4070318A50AA90303195D283221C63E37
:1000B00003185D280A3E03184028B71E6428A409C7
:1000C000A509A40A0319A50A240837290408A600CB
:1000D0003A0884008030B7050830A70003100318E1
:1000E000B70A8020A60CA70B6F280000AB1A370CAC
:1000F00080203A21031480202F08A3002E08D9283D
:100100008413AB1F8F28000838042B1F380680008B
:10011000841700083804031C380680009B28000858
:100120003804031C38062B1B380680008417380956
:1001300080059B2837172B081F39003EA1002A088D
:100140000E3E0318A10A371FE6283713A00002301D
:10015000F820E628B71329080319B7170530A800B7
:100160002730A3001030C0200330A300E830C020A7
:10017000A3016430C020A3010A30C0202408C7288E
:10018000A2002508A1002408A00016212008A00034
:10019000A8030319B71329080319D1282802031843
:1001A00008002008031DB713B71B0800303E322992
:1001B000A301A200FF30A207031CA307031C3729D9
:1001C0000330A100E630E620DA28A101FC3EA000C1
:1001D000A109031CF128FF300000A0070318EC2838
:1001E000A0076400A10FEB2808000310A10CA00CCD
:1001F000FF3E0318F52820083729A101A301A2001A
:1002000002300229A80023082102031D092922081F
:100210002002043003180130031902302805031DA1
:10022000FF3037290404031DFF303729A501A4013D
:100230001030A600210DA40DA50D2208A40223084C
:10024000031C230FA50203182C292208A407230846
:100250000318230FA5070310A00DA10DA60B1A2943
:1002600020083729840031088A003008820083136F
:10027000031383126400080083160A3099002430A7
:10028000980083129030980007309F00831606165E
:100290008616061786178615061405168515051089
:1002A000831205108316051085140515640083124A
:1002B00085185C2970295C29BE01BF016400051DF9
:1002C000662905148316051083126A290510831602
:1002D000051083125E296F300B206B300B20080055
:1002E00005148316051083120130A300F430D920C1
:1002F00005108316051083120130A300F430D920B5
:1003000005148316051083120120243C031D842943
:100310000120D9000120DA000120DB000120DC00EF
:100320000120DD000120DE000120DF000120E000CF
:100330000120E1000120E2000230A9000130B000FC
:10034000B1013220D8000120CE000430A9000130D4
:10035000B000B1013220C4002508C5000120CD0045
:100360000430A9000130B000B1013220C2002508DC
:10037000C3000120CF000120D0000120D1000120C6
:10038000CC000430A9000130B000B1013220C0001F
:100390002508C1000120D4000430A9000130B000BC
:1003A000B1013220CA002508CB000120D30004305F
:1003B000A9000130B000B1013220C8002508C900F1
:1003C0000120D5000120D6000120D7000120D20055
:1003D0000430A9000130B000B1013220C600250868
:1003E000C70064005A08493C031D4C2A05108316B7
:1003F000051083120130A300F430D92005148316B0
:100400000510433083120B204C300B2061300B2041
:100410004E300B205A300B2065300B2052300B2011
:1004200053300B2020300B2050300B2075300B2028
:100430006C300B2073300B2065300B2020300B20EC
:100440004D300B206F300B2074300B206F300B20A1
:1004500072300B2020300B2056300B2065300B20E3
:1004600072300B2073300B2069300B206F300B2063
:100470006E300B2020300B2034300B202E300B2020
:1004800030300B2020300B2032300B2030300B204E
:1004900030300B2037300B2064005A08573C031DC6
:1004A000DC2A0530BA000230B8005430AA00AB0193
:1004B000AE01AF0124306720590867205A08672031
:1004C0005B0867205C0867205D0867205E0867207E
:1004D0005F0867206008672061086720620867205E
:1004E0000230A9005808A400A5016630B000B1018F
:1004F000AA204E0867200430A9004408A40045083B
:10050000A5006630B000B101AA204D086720043074
:10051000A9004208A4004308A5006630B000B1015C
:10052000AA204F08672050086720510867204C0810
:1005300067200430A9004008A4004108A5006630E7
:10054000B000B101AA20540867200430A9004A086D
:10055000A4004B08A5006630B000B101AA205308E2
:1005600067200430A9004808A4004908A5006630A7
:10057000B000B101AA205508672056086720570827
:100580006720520867200430A9004608A4004708E5
:10059000A5006630B000B101AA200530BA000430D1
:1005A000B8005430AA00AB011120243C031DD42A0A
:1005B0001120D90059080B2064005A08523C031D31
:1005C000422C0530BA000230B8005430AA00AB010A
:1005D000AE01AF0124306720590867205A08672010
:1005E0005B0867205C0867205D0867205E0867205D
:1005F0005F0867206008672061086720620867203D
:100600000230A9005808A400A5016630B000B1016D
:10061000AA204E0867200430A9004408A400450819
:10062000A5006630B000B101AA204D086720043053
:10063000A9004208A4004308A5006630B000B1013B
:10064000AA204F08672050086720510867204C08EF
:1006500067200430A9004008A4004108A5006630C6
:10066000B000B101AA20540867200430A9004A084C
:10067000A4004B08A5006630B000B101AA205308C1
:1006800067200430A9004808A4004908A500663086
:10069000B000B101AA205508672056086720570806
:1006A0006720520867200430A9004608A4004708C4
:1006B000A5006630B000B101AA200530BA000430B0
:1006C000B8005430AA00AB011120243C031D642B58
:1006D0001120D9001120DA001120DB001120DC00EC
:1006E0001120DD001120DE001120DF001120E000CC
:1006F0001120E1001120E2000230A9001130B00009
:10070000B1013220D8001120CE000430A9001130F0
:10071000B000B1013220C4002508C5001120CD0071
:100720000430A9001130B000B1013220C200250808
:10073000C3001120CF001120D0001120D1001120C2
:10074000CC000430A9001130B000B1013220C0004B
:100750002508C1001120D4000430A9001130B000D8
:10076000B1013220CA002508CB001120D30004308B
:10077000A9001130B000B1013220C8002508C9001D
:100780001120D5001120D6001120D7001120D20051
:100790000430A9001130B000B1013220C600250894
:1007A000C70059080B205A080B205B080B205C0877
:1007B0000B205D080B205E080B205F080B206008F3
:1007C0000B2061080B2062080B200230A90058089A
:1007D000A400A5010A30B000B101AA204E080B20E8
:1007E0000430A9004408A4004508A5000A30B00060
:1007F000B101AA204D080B200430A9004208A40032
:100800004308A5000A30B000B101AA204F080B2010
:1008100050080B2051080B204C080B200430A90075
:100820004008A4004108A5000A30B000B101AA2088
:1008300054080B200430A9004A08A4004B08A50066
:100840000A30B000B101AA2053080B200430A900DF
:100850004808A4004908A5000A30B000B101AA2048
:1008600055080B2056080B2057080B2052080B2068
:100870000430A9004608A4004708A5000A30B000CB
:10088000B101AA205A08A0005030FD20B2005A0839
:10089000A0005130FD20B400320884003408122139
:1008A000B400B5006400340835040319EA2C05309F
:1008B000BA000230B8005430AA00AB01AE01AF015B
:1008C00024306720590867205A0867205B08672092
:1008D0005C0867205D0867205E0867205F08672066
:1008E0006008672061086720620867200230A9005D
:1008F0005808A400A5016630B000B101AA204E0836
:1009000067200430A9004408A4004508A50066300B
:10091000B000B101AA204D0867200430A9004208A8
:10092000A4004308A5006630B000B101AA204F081A
:10093000672050086720510867204C086720043062
:10094000A9004008A4004108A5006630B000B1012C
:10095000AA20540867200430A9004A08A4004B08C4
:10096000A5006630B000B101AA205308672004300A
:10097000A9004808A4004908A5006630B000B101EC
:10098000AA20550867205608672057086720520894
:1009900067200430A9004608A4004708A500663077
:1009A000B000B101AA200530BA000430B8005430BC
:1009B000AA00AB011120243C031DDA2C1120D90020
:1009C0000430A9005908A400A5010A30B000B10103
:0609D000AA20D32C8429AB
:02400E002A3F47
:00000001FF
